:030000000219FDE5
:03000B000200AA46
:03002B0002015F70
:03005B000202F5A9
:030073000202DBAB
:1000800002030406080C10182030406080040608A3
:100090000C10182030406080A0C000070F1F3F0DDB
:1000A0000D0403060D0502030202C2AFC0D0C0E07A
:1000B000206217E5256002E473E525F4F58A758B67
:1000C00000D262D0E0D0D0D2AF3285268AC262E5BB
:1000D00026F4602F758B00D0E0D0D0C290C291C2C0
:1000E00092D2AF32C290C291C292206E0C206609A9
:1000F0007405D5E0FDE57E4290758B00D0E0D0D050
:10010000D2AF32758A00C28DD26201F901B930686E
:1001100005206602D29001B9306805206602D291AE
:1001200001B9306805206602D29201B9C2953068E3
:100130000A2066077432D5E0FDD29001B9C294302E
:10014000680A2066077432D5E0FDD29101B9C293E6
:1001500030680A2066077432D5E0FDD29201B9C238
:10016000AFC2AD53E6EFC0D0C0E0D2D3D2AFC2CE63
:10017000E52A6007207449152A21C07800790020FB
:10018000742EE580307E01F430E60278FF53DACF3A
:10019000207E0343DA20307E0343DA10C2D8C271D6
:1001A000E580307E01F430E60279FFC3E89970CB38
:1001B000306103752A40207403752A40885FD2702D
:1001C00020740DE52B6004152B21D043DA01C2D831
:1001D00020700221E3A85F206102C2702074022116
:1001E000E188227882B60403852224C3E525944061
:1001F0004002D26420CF0AD0E0D0D043E610D2AD86
:1002000032C2CF053A7802E52A6005307402152A19
:10021000C3E55F94014005756200412D756300756B
:100220006C00E5622401F56250037562FF7982B7C4
:10023000020D306D1DC3E52294324016854D2279A2
:1002400082B7030E306D0BC3E52294324004798EE1
:100250008722C3E5239522600840041523416105E8
:1002600023D8CA056CE56C7002156CD56D63756D8D
:10027000017805C3E56C956E4057C3E56C956F50EA
:10028000087801756D03020295C3E56C9570500501
:100290007801756D01C3E5659524401E7982B70428
:1002A0000241C6206D14852465E56C046003856EEB
:1002B0006C756D0175233C0202D1E565285005750A
:1002C00065FF41C6F565E5650470067563FF756CED
:1002D000FFD0E0D0D043E610D2AD32C2AFC0D05391
:1002E000E67FC26075910085569485579575910497
:1002F000D0D0D2AF32C2AF53E6EFC2ADC0D0C0E073
:10030000C0F0D2D3D2AFA8FBA9FCC2D83071026131
:100310005C53DACF207E0343DA10307E0343DA20C9
:10032000D271E580307E01F420E6026133882789AE
:1003300028A14153DACF207E0343DA20307E0343E5
:10034000DA10C2D8C271307402A12D7800E5803075
:100350007E01F430E602A12D885FA11553DACF208B
:100360007E0343DA20307E0343DA10C2712061023B
:10037000813553DACF207E0343DA10307E0343DA2F
:1003800020C2D8D271885A895BC3E89558F8E9959C
:1003900059F97B007E087A00C3E8948CE9940050F8
:1003A00005755E008127882178A2E6A8216055C3E3
:1003B000E894C8E994005008E4D2E4FB7A0A810288
:1003C000C3E89468E994015008E4D2E3FB7A0F8112
:1003D00002C3E894D0E994025008E4D2E2FB7A1E0A
:1003E0008102C3E894A0E994055008E4D2E1FB7AC5
:1003F0003C8102C3E89498E994085008E4D2E0FBF9
:100400007A787E00C3E8955CFCE9955DFD30E70AEB
:10041000ECF42401FCEDF43400FD755E00C3EC9AAD
:10042000ED9E5003755E01885C895D855A58855B39
:10043000597802A115C3E89527F8E99528F9307C89
:100440000281F9307B0281F9307A0281F220750253
:100450008158E9FDE8FC8177E9C313F9E813F83026
:10046000790281F2E9C313F9E813F830780281F2D6
:0F047000E9C313FDE813FC20612CC3EC941CEDD1
:10047F0094024002818EED701EC3EC94C850180593
:10048F0029E52970021529C3E529940A5002A12DE7
:10049F00755F00D270A12DE5296002152974002027
:1004AF007F037896E624FAFEE43400FFC3EC9EFC4B
:1004BF00ED9FFD50067800790081F9C3EC94FFEDB4
:1004CF009400400678FF790081F9EC8575F0A4C59A
:1004DF00F0A2F733F87900400302051578FF790091
:1004EF00020515E9C313F9E813F8307C0EE9600231
:1004FF0078FFC3E81338F8E43400F9C3E894FFE950
:10050F009400400278FF885FD270206102A12D74A1
:10051F001FF4552F4BF52FC274EB7002D274752A4E
:10052F0040307403752A0A306102A14120740353CD
:10053F00DAFE207403752B20D0F0D0E0D0D0D2ADEE
:10054F0043E6103279010205717903020571790AC8
:10055F00020571791E020571796402057179C8026D
:10056F0005717817E4D5E0FDD8FAD9F6227A147B15
:10057F00780205987A107B8C0205987A0D7BB4026D
:10058F0005987A0B7BC80205987902B27DE4C29474
:10059F00D5E0FDD291D5E0FDC291D5E0FDD294D545
:1005AF00E0FDD290E576D5E0FDC2907496D5E0FDE2
:1005BF00D9D9EAF8D5E0FDD8FBDBCEC29422C37CB3
:1005CF00007D0075F00005F0EA33FAEB33FB50F6CF
:1005DF00EB13FBEA13FAC3E9FFE8FEE89AF8E99B8D
:1005EF00F95004EFF9EEF8B3EC33FCED33FDD5F031
:1005FF00DFEDF9ECF822E889F08A20D2D4F8A9F0DF
:10060F007B0030F70B7BFFF42401F8E9F43400F999
:10061F00E88520F0A4ADF0F8E98520F0A4AFF0FE56
:10062F00ED2EF974003FFA7C04C3EA13FAE913F9CB
:10063F00E813F8DCF48BF030F70AE8F42401F8E95A
:10064F00F43400F9E889F0C2D4F8A9F0227882B620
:10065F0004030206FBC3E55F9419401EE52D540603
:10066F007018206D3678057994E7146007780A14AE
:10067F0060027812C3E54198401F306D09856765A8
:10068F00756CFF756D01852224E4F545F546F54738
:10069F00F548F549C26D0206FBD26D7994E71470E7
:1006AF0013E523F43333F913F8E9540104F9E8544B
:1006BF00FE0206EFE714147014E523F4333333F915
:1006CF0013F8E9540304F9E854FC0206F7E523F4A0
:1006DF0033333333F913F8E954070404F9E854F8C2
:1006EF00C39440F8E99400F98845894622C3E5414F
:1006FF0013F9E54013F8C3E54598F8E54699F95025
:10070F000CC3E89480E994FF4016020733C3E894C2
:10071F007FE994005003020733787F790002073393
:10072F00788079FF884A894B22E54A2547F8E54BBF
:10073F003548F9854B20E4300701F43549FA30E7A5
:10074F0009C3EA94F04015020771C3EA940F5003EE
:10075F0002077178FF79FF7A0F020771780079002D
:10076F007AF0C3E5249564500AC374019524500BA5
:10077F0002078FE54B20E70E02078FE54B30E706A8
:10078F00884789488A492278A4E6FAC3E54A33F8AC
:10079F00E54B33F9D105E930E70BC3E89480E994D1
:1007AF00FF4013E1C9C3E8947FE994005002E1C907
:1007BF00787F7900E1C9788079FFE820E715C3E5F4
:1007CF002398F84009C3E8940140030207F0780129
:1007DF000207F0E8F424012523F840030207F0781C
:1007EF00FF884C2278A5E6FAA848A949D105E93037
:1007FF00E70CC3E89401E994FF4016020824C3E80C
:10080F0094FFE99400500302082478FF790002084E
:10081F0024780179FFE920E715C3E54C98F84009E2
:10082F00C3E89401400302084B780102084BE8F437
:10083F002401254CF8400302084B78FF88242278C6
:10084F00FFC26420693D206A12D264C3E541940A55
:10085F004009C3E52594405002C26479A1E76023A3
:0D086F00E541601F74FF8541F0848539F07C
:10087C00306A0375F005A4F8C5F0600278FFC3E890
:10088C0095675002A867886622C3E5409440E5410D
:10089C009401E56650031401A6046002F566227803
:1008AC0083E6F520120F4575E89012055375E89014
:1008BC00E5E820ECFBA8BDA9BE120FDF7571987599
:1008CC007200C3740013FD7498606613FC74982C4A
:1008DC00FC74003DFDECFAEDFBC3E89AE99B401477
:1008EC00E5712498F571E5723400F572EA2CFAEB97
:1008FC003DFB80E5AE71AF72C3E57213F9E5711380
:10090C00F8C3E913F9E813F87A03C3E913F9E81308
:10091C00F8DAF7AA201A70097571007572000209CD
:10092C003D1AEA6008EE28FEEF39FFDAF88E718F77
:10093C00722275E890227883E6FFE5E820ECF7A8B0
:10094C00BDA9BE0573C3E57394084052757300E9E5
:10095C00FA79A0E76044EA7007E574601B02097835
:10096C00C3E895746010E5745006600C1402098499
:10097C000460F9020984E574F574C3946D401B7529
:10098C0064C0C394044013756480C39404400B7515
:10099C006440C39404400375640075BB0E22EFC31E
:1009AC009401601F7498601BC3E894FFE994035092
:1009BC0012C3E89571E995725009E564600C1564F1
:1009CC000209D6E564F460020564A864C3E52498C2
:1009DC005002A824C3E89565400AA865E565F46053
:1009EC000385656488258826E573B4070375BB10F9
:1009FC0022743279A687F0A4C5F0A2F733F8C3E8C5
:100A0C0095644002A86488228824882588268867F3
:100A1C00227540007541F022C2AF75C820A8CCA940
:100A2C00CDAA3A30CF010A75C824D2AFAB3BAC3C4F
:100A3C00883B893CC3E89BF8E99C206908F930673E
:100A4C000261394196AD3D8A3DF9EA9DFA60047820
:100A5C00FF79FFAE3EAF3F8B3E8C3FC3EC9FFCC398
:100A6C00E99CF542A83BA93CC3E89EF8E99FF9C371
:100A7C00E54113FBE54013FAE82AF540E93BF54163
:100A8C0050067540FF7541FF41E0AA40AB41AC40B8
:100A9C00AD417E047F02C3EB940440021E1FC3EBE6
:100AAC00940840021E1FC3ED13FDEC13FCDEF7C3CC
:100ABC00EA9CFAEB9DFBEF6009C3E913F9E813F824
:100ACC00DFF7EA28FAEB39FB8A408B4150067BFFB3
:100ADC008B408B41C3EB94025002D2673069047F88
:100AEC0003610B7892E6FFC3E537948240110FC384
:100AFC00E53794A040010FC3EF940640027F057EBA
:100B0C0007E541C4540FF9E541C454F0F8E540C47D
:100B1C00540F28F8C3E89EFAE99400FB4009C3EA95
:100B2C009402EB940050047A02E4FB6185AA40AB7A
:100B3C0041EBC4FEEAC4540F4EFCC3EA9CFAEB949E
:100B4C0000FBC3E813C313F8EA28FAEB3400FB8A62
:100B5C00408B41C3EB94024002C2677807EBC4FEA2
:100B6C007B00EAC4540F4EFAC3EA98FA4005C394CA
:100B7C000250027A027892E6FF306002618585525B
:100B8C0056855357D26043E680C3E49AF8E49BF948
:100B9C00306702811FE8FAE9FBD3E913FDE813FC87
:100BAC0088528953C3EF94036038EF20E00DE82C92
:100BBC00F8E93DF9ECFAEDFB020BDAE828F8E93933
:100BCC00F9C3E82402F8E93400F97AFE7BFFC3EF9D
:100BDC009403400E8A548B55884E894F8C508D51FE
:100BEC008153885489558A4E8B4F8C508D51306966
:100BFC0020C3E53394034019E542A2E713F8E55509
:100C0C00F4240138400B20E7087554FFF42401F557
:100C1C00558153E8FAD3E813FC8852C3EF94036070
:100C2C0020EF20E007E82CF8ECFA813FE8282402BA
:100C3C00F87AFEC3EF940340088A54884E8C508196
:100C4C005388548A4E8C50E56BC3335002646BF559
:100C5C006B306002815D753402D26043E680E52D15
:0F0C6C0054066026A840A941C3E913F9E813F81C
:100C7B00C2AF53E67F759100C3E498F594E499F500
:100C8B0095759104D26043E680D2AF22D26575444C
:100C9B0000752000306B03752040020CB6D26575D1
:100CAB004400752040306B03752000D2AF780120D3
:100CBB006722E52D54066002C265C3E541940540E9
:100CCB0013780294054008780394054002780630A7
:100CDB006902780A206019E544601530690AC3E59A
:100CEB003394034003D53406D2AFD26CA1889165FF
:100CFB00D2AF0000C2AF206726E541C3FB940F4083
:100D0B00027B0FEB240530730123306A0274282019
:100D1B00620123F93069027982E58BC39940B505ED
:100D2B0044E59BF45440B52002A17230690A08C314
:100D3B00E8940A40010881DF20650281B6C2655341
:100D4B00E67F7591003067107594007595FE75916F
:100D5B0004D26043E68081B6AE40AF41C3E49EF55A
:100D6B0094E49FF595A159C3E5339402500281B6E3
:100D7B0030650281B6D802A18681DFC26C53E67F53
:100D8B00759100855494855595759104854E5685BE
:100D9B004F57D26043E680D2AFE52D540660082052
:100DAB006A020533020DC2306C0D206B0A206507F9
:100DBB001581158102161222780030640530650208
:100DCB007801E53775F007A4F9E5F028F5F0E9A20D
:100DDB00F013A2F113A2F213F537C39478500375F5
:100DEB003778C3E53795384008D266C290C291C2B6
:100DFB0092306002A1FC855056855157D26043E674
:100E0B008022207D11C2AF754302C294D295D2AF1E
:100E1B00759F10020FDCC2AF754302C294D293D2FE
:100E2B00AF759F10020FDC307243207D20C2AF756F
:100E3B00430390013D757E10C292C293306204D27F
:100E4B0091C150D294D2AF759F20020FDCC2AF7507
:100E5B00430390013D757E10C290C295306204D25F
:100E6B0091C170D294D2AF759F00020FDC207D1719
:100E7B00C2AF754303900118C292306202D291D275
:100E8B00AF759F20020FDCC2AF754303900118C2F0
:100E9B0090306202D291D2AF759F00020FDC207DA1
:100EAB0011C2AF754304C295D293D2AF759F0002A6
:100EBB000FDCC2AF754304C293D295D2AF759F209E
:100ECB00020FDC307243207D20C2AF7543059001C9
:100EDB002C757E20C291C294306204D290C1ECD2A8
:100EEB0095D2AF759F10020FDCC2AF754305900111
:100EFB004E757E08C291C294306204D292E10CD23C
:100F0B0093D2AF759F10020FDC207D17C2AF7543D4
:100F1B000590010EC291306202D290D2AF759F1034
:100F2B00020FDCC2AF754305900122C2913062EB18
:100F3B00D292D2AF759F10020FDC207D11C2AF751C
:100F4B004306C293D294D2AF759F20020FDCC2AF7F
:100F5B00754306C295D294D2AF759F00020FDC3059
:100F6B007242207D20C2AF75430190014E757E0801
:100F7B00C290C295306204D292E188D293D2AF75FF
:100F8B009F00020FDCC2AF75430190012C757E20D0
:100F9B00C292C293306204D290E1A8D295D2AF75BF
:100FAB009F20E1DC207D16C2AF754301900122C268
:100FBB0090306202D292D2AF759F00E1DCC2AF7566
:100FCB00430190010EC292306202D290D2AF759F54
:100FDB0020C2662290010C757E00C290C291C29213
:100FEB00C295C294C293C2622278807607087607B4
:100FFB000876010876040876FF0876FF08760B085A
:10100B007602087601087601788C7601087600085E
:10101B0076B40876FF0876FF0876FF087603087625
:10102B00FF0876010876FF0876250876D0087678D3
:10103B000876C80876040876FF087601087600085B
:10104B00767A087607087601087601087600087626
:10105B00FF227887E6FFC2727888C27DE630E10214
:0E106B00D27DC27E7889E630E102D27EC3EFEC
:1010790094026008758E01D27302108A758E00C2BF
:1010890073227880E6149000809378A4F67881E63C
:10109900149000809378A5F67886E61490008D93D5
:1010A90078A6F6789FE6F8700108C3E89411400223
:1010B9007811E82828F56E256E256E28F56F256EBE
:1010C9002828F570789CE67538FF75390CB4020646
:1010D9007538A075390AB4030675388275390578EB
:1010E900A3E61490009A93F569120FDF22227896ED
:1010F900E6FA7897E6FB7888E6B40305C3EB940E25
:10110900FB307F047A007BFFC3EB9AFCC3948250C7
:10111900027C827575000575EC8575F0A4C3E5F050
:10112900947D40F222D27F11F71205627A007B008A
:101139007C10120558E55F2AFA74003BFBDCF37C4E
:1011490004C3EB13FBEA13FADCF7FEC27F11F722A3
:10115900E5EF20E6037520000520903FFFE5201408
:101169006006901DFF1460009304600375EF12532D
:10117900D9BF7581C043FF8012055375EF0243B291
:1011890003E5B3240420E70DF521E5E320E0068516
:1011990021B343E301120FDF7580FF75A40075F1D8
:1011A900D475D4BF75904075A53F75F23F75D500CC
:1011B90075A60175E241E4F8F6D8FD756B01120FC9
:1011C900F412165A78988676753001C2AF12056CFA
:1011D90012057C12056212058312056212058A1234
:1011E900056212177D12056C12056C120567C2AFF4
:1011F90078FA79FA308607D9FBD8F7021C00115D15
:10120900118B11F611F778988676120FDF758850D1
:1012190075891275C82475910475D84075A8227509
:10122900B80275E690759B80759D0075D10E75BCE9
:101239005875BB0E75BA1175E880120553D2AF12F5
:1012490008AB53DACF207E0343DA20307E0343DA3A
:101259001043DA01C2D8C27112056CD2617B037ADC
:101269000CE55E70077A0CDB030211F712056220A8
:1012790070030211F7C270E55FC3940240E1E52FE4
:10128900541F856160F561B560D5DAD5C26153DA5D
:10129900CF207E0343DA20307E0343DA10C2D8C25E
:1012A9007178A2E67008D274E52F54E0F52FC27563
:1012B900752900120567307409C3E529940A4002AB
:1012C900D27512055878023074027800C3E55F9828
:1012D90040F0C2AF12057C12057C12057CD2AF1218
:1012E900056C754D00120558788CE6C394015003BE
:1012F9000213C4E530C3940150030213C4207435AA
:10130900C3E55F94FF50030213C4C2AF120591D223
:10131900AF120567C3E55F940150EFC2AF12057CB8
:1013290012055D12057CD2AF120567C3E55F94FF14
:1013390040E90218027F05D27F11F7120567C2AF93
:10134900C27F11F7AE5FC3E55F947FD2AF407612DB
:101359000553C2AF120591D2AFDFDC312EC3EE9433
:10136900057897F612056C12169C1217857F0AD21A
:101379007F11F7120567C2AFC27F11F7AE5FC3E5F0
:101389005F947FD2AF50E6120553C2AF12057C12AB
:10139900055D12057CD2AFDFD6312EEE2405789695
:1013A900F612056C12169C1217B412056711F7C3D1
:1013B900E55F94FF50026106021802C3E55F954D8F
:1013C9004003855F4D12056778017988E7B4030208
:1013D9007805C3E55F98400241EEC2AF120591124C
:1013E9000591120591D2AF12056C753000E4F53103
:1013F900F5320531E531F470390532789AE6781914
:10140900146012783214600D787D14600878FA142B
:101419006003753200C3E53298401715327531B44F
:1014290078998676C2AF120591D2AF7898867612EE
:10143900056712055DE52A700530740221F7780108
:101449002074027806C3E55F9840A7120567E52A6C
:1014590070030211F7C2AF120FDFE4F522F523F58D
:0E14690024F525F526F56AD2AF7885E6C33363
:10147700F568E4F545F546F547F548F549F573F59B
:101487002CF52DF53775730875BB10120553120926
:101497003EE5E820ECFBA8BDA9BEE97001F8887419
:1014A70012094275730875BB107887E6FE7602113C
:1014B7005D7887EEF6C2AF7564FF1209FD85226479
:1014C700852265852266D2AF7522017524017525AF
:1014D7000175260185636C756D017888E6B403078D
:1014E700C27D307602D27DD268D269753300120F81
:1014F70045120F6A120A1D120A24120A1D120A2423
:10150700120A1D021519C2AF115DD2AF75730075AE
:10151700BB0E120CA812065C120DC3120E0D120A96
:1015270024120C97306D031206FC20670312084E35
:10153700306703120895120DC3120E32120A2412D5
:101547000CA8306D03120738120DC3120EA9120A28
:1015570024120C97306D03120796120DC3120ECE8C
:10156700120A24120CA8306D031207F3120DC312CE
:101577000F45120A2412093E120C97120DC3120FBF
:101587006A120942120A2430692F206B2C8567647E
:1015970085676585636C756D0179187A0CC3E533CA
:1015A700994009C269D26A8A350215C0C3E55F94BA
:1015B70001400302151902161A306A1B206B18E541
:1015C70035147004C26AA10DF535C3E55F94014077
:1015D7000302151902161A753600C3E56294014015
:1015E7000985676585636C756D01C3E56278FA984F
:1015F7005021307404E52A601A78F0306B0585674E
:10160700647820C3E541985002A1190536E55F606B
:1016170002C11D753600C2AF120FDF7887E6FE766E
:1016270002115D7887EEF6E4F522F523F524F5251A
:10163700F526F568C268D2AF120553120FDF307472
:1016470006E52A700221F7788DE6C394014002412E
:10165700CB61F6901A0D78201216DEE520B4A50CA2
:10166700A31216DEE520B45A0302167C120FF412F9
:10167700169C02169B901A0378807B0A1216DEA32B
:1016870008DBF9901A0F788C7B181216DEA308DB9B
:10169700F9901A2722C2AF12171D1216F7901A00D7
:1016A700740E1216E3A374041216E3A3741412162D
:1016B700E3901A0378807B0A1216E2A308DBF990FD
:1016C7001A0F788C7B181216E2A308DBF912173071
:1016D70012170E901A2722E493F622E6438F01533E
:1016E7008FFD75EF0275B7A575B7F1F0538FFE2221
:1016F700438F02438F0175EF0275B7A575B7F19058
:101707001A0DF0538FFC22901A0D74A5D1E3901A8D
:101717000E745AD1E3227A3079D07820901A40D1CA
:10172700DEE520F709A3DAF7227A3079D0901A405C
:10173700E7D1E309A3DAF922AB77A878BB010279ED
:1017470080BB02027981BB03027982BB04027994D0
:10175700BB05027983BB06027986BB07027992BB78
:1017670008027987BB0902799CBB0A027988BB0BFF
:10177700027989E8F7227C0512056CDCFB22C2AFEF
:1017870012057C12058312058A12059112055D1256
:10179700057C12058312058A12059112055D120553
:1017A7007C12058312058A120591D2AF22C2AF12AD
:1017B700059112058A12058312057C12055D120533
:1017C7009112058A12058312057C12055D12059197
:1017D70012058A12058312057CD2AF22AE77AF7845
:1017E700C2AF12057C12057C12057C12055DDEF284
:1017F70012059112055DDFF8D2AF22121785121775
:101807007D12177D7577017578017579001217E3D9
:101817007C05AD5F12056CC3ED955F70F5C3E55FA1
:101827009401400AC3E55F94FF4037021846121738
:101837003F12169C121785C2AF75EF1212177DDC87
:10184700D10579C3E5799403500280C112177D054C
:1018570078E5771490009F93F808C3E578985002CD
:0F18670080A812177D12177D0577C3E577940CC3
:1018760050028094120FF412169CC2AF75EF12122A
:02188600177DCC
:0319FD000211597B
:101A00000E041407070104FFFF0B020101A55A0190
:101A100000B4FFFFFF03FF01FF25D078C804FF01DA
:081A200000FF07010100FFFFB8
:101A400023524354696D65723641232020202020A3
:101A500023424C48454C4923463333302320202031
:101A60002020202020202020202020202020202076
:101C0000C2AFC2D353D9BF7581C043B20343FF8073
:101C1000752438752503B1C975EF0275E24043F1AB
:101C20004053A4BF75D400D2867DFA780379E67C50
:101C300010752200752300901DD67B0675249875BB
:101C400025013086028142208608D8FBD9F9DCF7CD
:101C500081B4308608D8FBD9F9DCF781B4B189E4C6
:101C600093A3C39A6004DDC381B4DBDBB17B600264
:101C7000812B7B08E493FAA3B15CDBF87A30B15C8A
:101C8000752200752300B17BEAFCEBFDC3ED94FEE9
:101C9000400EB17B8A278B28ED30E0048A828B834B
:101CA000B17B7AC270D8C3ED94FE601350CEBD00F4
:101CB00025EC60097520007521FF0200008100A855
:101CC00027A9280809D804D90281D3B17FEA89AAB3
:101CD000F281C50D81A0C3ED94035049EDA2E092BD
:101CE000007AC5C3E5829400E583941C50902000DF
:101CF00010438F02438F0175B7A575B7F1F030001F
:101D00001FA827A9280809438F01538FFDD804D99C
:101D100002A12089AAE275B7A575B7F1F0A3A10DBC
:101D2000538FFC817C7AC1BD030CE493A3FAB140CC
:101D3000DCF8B138817C817EAA22AB23B15CEBFA5E
:101D4000EA6222752608C3E52313F523E52213F57D
:101D50002250066323A0632201D526EAB1C9B1C986
:101D600075260AEAF4200102D286300102C286B149
:101D7000C9C3134002C201D526EB22B17FEAFB2082
:101D80008602A17F308602A184752608AE24AF2585
:101D9000C3EF13FFEE13FEB1CDB1C9C3EA13308612
:101DA000024480FA30E703632201C3E52313F523DD
:101DB000E52213F52250066323A0632201D526D91C
:101DC000E52265236523F52222AE24AF250E0FDE22
:101DD000FEDFFCD20122424C48656C693437316326
:041DE000F3300601D5
:00000001FF
